:0200000480007A
:1000000013058000731005021305400073101502DC
:10001000731040F17310103037F1FF7FEF00801E36
:10002000EF10D00873000000938B0600130D07003B
:10003000130F01009303050013051000635C7500A6
:1000400013010180130305006B5003001305150015
:100050006FF0DFFE1300000013000000130000002B
:1000600013000000130000001300000013010F0034
:1000700013050000930F0600938D0300130000008A
:100080001300000013000000130000001300000024
:10009000130000001300000013000000EBE0BF019C
:1000A0001300000013000000130000001300000004
:1000B0001300000013000000170500001305451B86
:1000C0006B40050017030000130343F66B000300A9
:1000D000678000001702000113028225232002001E
:1000E0002322120023242200232632002328420048
:1000F000232A5200232C6200232E72002320820226
:10010000232292022324A2022326B2022328C2021F
:10011000232AD202232CE202232EF20223200205FC
:1001200023221205232422052326320523284205F3
:10013000232A5205232C6205232E720523208207D1
:10014000232292072324A2072326B2072328C207CB
:10015000232AD207232CE207232EF20713021000D2
:1001600067800000170200011302821C03200200B6
:1001700083204200032182008321C2000322020166
:1001800083224201032382018323C201032402024A
:1001900083244202032582028325C202032602032E
:1001A00083264203032782038327C2030328020412
:1001B00083284204032982048329C204032A0205F6
:1001C000832A4205032B8205832BC205032C0206DA
:1001D000832C4206032D8206832DC206032E0207BE
:1001E000832E4207032F8207832FC20713020000CA
:1001F00067800000732500026780000073251002ED
:1002000067800000130101FE232E1100232C8100C2
:1002100013040102232604FE6F0040030327C4FEDB
:10022000B7170000938747973307F702B707008196
:100230009387C742B307F70013850700EF00C04359
:100240008327C4FE938717002326F4FE0327C4FEEA
:100250009307F001E3D4E7FC130000008320C10101
:10026000032481011301010267800000130101FDD5
:1002700023261102232481022322A1031304010354
:100280001300000013070D00B7170000938747976E
:100290003307F702B70700819387C742B307F70018
:1002A00013850700EF00005093070500638A0702DB
:1002B00013070D00B70700811317270093874728FE
:1002C000B307F7001307100023A0E70093070D0002
:1002D00063960700EFF01FE96F00C0057300000090
:1002E00013070D00B7170000938747973307F702EE
:1002F000B70700819387C742B307F700130784FD50
:100300009305070013850700EF00C03F832704FE15
:10031000138107008327C4FD832584FD032644FE43
:10032000832684FE0327C4FE13850700EFF0DFCF8A
:10033000730000008320C10203248102032D4102C7
:100340001301010367800000130101FB2326110440
:100350002324810413040105EFF0DFE92324A4FE24
:1003600093090100930710002326F4FE6F00C008D4
:100370000327C4FEB7170000938747973307F70298
:10038000B70700819387C742B307F70013850700BB
:10039000EF00404193070500639A07040327C4FE5A
:1003A000B7170000938747973307F702B707008115
:1003B0009387C742B307F700130704FD93050700AF
:1003C00013850700EF000034832784FD13810700A5
:1003D000832744FD832504FD0326C4FD832604FEF4
:1003E000032744FE13850700EFF0DFCD8327C4FE0B
:1003F000938717002326F4FE8327C4FE032784FE79
:10040000E3E8E7F613810900EFF0DFCC9307020081
:1004100063880704B70700811385C742EF0080385F
:1004200093070500639E0702930784FB93850700EB
:10043000B70700811385C742EF00C02C832704FC57
:10044000138107008327C4FB832584FB032644FC18
:10045000832684FC0327C4FC13850700EFF0DFBC70
:10046000130000008320C10403248104130101054B
:1004700067800000130101FB23261104232481045B
:1004800013040105232EA4FA232CB4FA232AC4FA58
:100490002328D4FAEFF01FD7EFF0DFD52322A4FEF4
:1004A00013090100232604FE232404FE6F00000923
:1004B000B709FFFF33013101832784FE2326F4FCB3
:1004C000832784FB2328F4FC93070100232AF4FCF0
:1004D000832744FB232CF4FC832704FB232EF4FC0A
:1004E0008327C4FE2320F4FE0327C4FEB7170000B1
:1004F000938747973307F702B70700819387C7426F
:10050000B307F7001307C4FC930507001385070022
:10051000EF00C0188327C4FE938717002326F4FE3C
:100520008327C4FE032744FE63E4E700232604FE7A
:10053000832784FE938717002324F4FE032784FE79
:100540008327C4FBE366F7F613010900EFF0DFDF52
:10055000130000008320C10403248104130101055A
:1005600067800000130101FD23261102232481026C
:1005700013040103232EA4FC8325C4FDB7070081C7
:1005800013850704EF000035EFF0DFC62320A4FE3B
:10059000232604FE6F004006232604FE232404FEC7
:1005A0006F00C003B7070081032784FE13172700DD
:1005B00093874728B307F70003A7070093071000A6
:1005C0006318F7008327C4FE938717002326F4FEE1
:1005D000832784FE938717002324F4FE032784FED9
:1005E0009307F001E3D0E7FC8325C4FEB707008141
:1005F0001385C704EF00002E0327C4FE8327C4FD24
:10060000E31CF7F8232204FE6F008002B707008185
:10061000032744FE1317270093874728B307F700E3
:1006200023A00700832744FE938717002322F4FEAC
:10063000832744FE032704FEE3EAE7FC13000000DF
:100640008320C1020324810213010103678000009B
:10065000130101FF232681002324710113040101EA
:1006600093870B00138507000324C100832B8100AF
:1006700013010101678000009302050013030000CD
:100680009303700023A0620023A2620023A46200EF
:1006900023A6720023A86200678000009302050071
:1006A00003A382001303130023A4620013834201F7
:1006B00083AE420093935E003303730003AE0500E4
:1006C0002320C30103AE45002322C30103AE8500EE
:1006D0002324C30103AEC5002326C30103AE0501D5
:1006E0002328C30103AE4501232AC301938E1E00B4
:1006F000130F20036394EE01930E000023A2D20196
:10070000678000009302050003A38200130000002D
:10071000130000001300000013000000130000008D
:10072000130000001303F3FF23A4620013834201AC
:1007300083AE0200930F2003138F0E00130F1F00D0
:100740006314FF01130F000023A0E20193935E00E6
:1007500033037300032E030023A0C501032E4300BF
:1007600023A2C501032E830023A4C501032EC300C9
:1007700023A6C501032E030123A8C501032E4301AF
:1007800023AAC501678000009302050003A382002D
:1007900013050000130E200363146E0013051500EB
:1007A000678000009302050003A382001305000088
:1007B000130E000063146E0013051500678000001F
:1007C0009302050003A3C20083A3020133B56300B3
:1007D00067800000130141FF232011002322B10094
:1007E0008345050063880500EF00C001130515006F
:1007F0006FF01FFF83200100832541001301C1001A
:1008000067800000B708010023A0B80067800000DF
:10081000130101FD23261102232481021304010385
:10082000232EA4FC0327C4FD9307F00063E4E70232
:10083000B70700810327C4FD131727009387471CC0
:10084000B307F70083A7070013850700EFF09FF8B1
:100850006F004007930700022326F4FEA30504FE61
:100860008327C4FE9387C7FF0327C4FDB357F70050
:1008700093F7F7002322F4FE832744FE63860700E4
:1008800093071000A305F4FE8347B4FE63820702BA
:10089000B7070081032744FE131727009387471CDF
:1008A000B307F70083A7070013850700EFF09FF257
:1008B0008327C4FE9387C7FF2326F4FE8327C4FE45
:1008C000E340F0FA8320C1020324810213010103F3
:1008D00067800000130101FE232E1100232C8100EC
:1008E000130401022326A4FE2324B4FE0325C4FE20
:1008F000EFF05FEE032584FEEFF09FF1B707008174
:1009000013854709EFF01FED130000008320C1019C
:10091000032481011301010267800000130101FD1E
:10092000232611022324810213040103232EA4FC95
:10093000232CB4FC232AC4FC2328D4FCB7670281EF
:100940000327C4FD23AAE71CB76702819387471DCD
:10095000032784FD23A2E700B76702819387471D21
:10096000032744FD23A4E700B76702819387471D4F
:10097000032704FD23A6E700EFF05F882324A4FEED
:10098000032704FD832784FEB357F7022326F4FED2
:10099000032704FD832784FEB377F70263880700EB
:1009A0008327C4FE938717002326F4FEB7670281CE
:1009B0009387471D0327C4FE23A8E700032704FDF0
:1009C000832784FE6362F702B76702819386471D1F
:1009D000B7170080138607A4832584FE032504FD32
:1009E000EFF05FA96F000002B76702819386471D91
:1009F000B7170080138607A4832504FD032504FD93
:100A0000EFF05FA7EFF00FFF2322A4FE032704FD02
:100A1000832744FE63F8E700032544FEEFF09FB40C
:100A20006F00C000032504FDEFF0DFB313000000EA
:100A30008320C102032481021301010367800000A7
:100A4000130101FA232E1104232C8104130401063F
:100A50002326A4FA2324B4FAEFF09FBF232CA4FC8E
:100A6000832784FD83A70700232AF4FC832784FDC2
:100A700083A747002328F4FC832784FD83A78700EE
:100A80002326F4FC832784FD83A707012326F4FE95
:100A90000327C4FE8327C4FAB307F7022324F4FE16
:100AA0008327C4FE639A0700930710002326F4FEF1
:100AB0008327C4FA2324F4FE832784FD83A7C70079
:100AC0002324F4FC232204FE6F00800D232004FE67
:100AD000232E04FC6F008007032784FA832784FCFD
:100AE000B307F7020327C4FDB307F7002322F4FC82
:100AF000032784FC8327C4FDB307F702032784FE82
:100B0000B307F7002320F4FC832744FC93972700C6
:100B1000032744FDB307F70003A70700832704FC5E
:100B200093972700832604FDB387F60083A7070069
:100B3000B307F702032704FEB307F7002320F4FEF0
:100B40008327C4FD93871700232EF4FC0327C4FDDD
:100B5000832784FCE362F7F8032784FA832784FC65
:100B60003307F702832784FEB307F700232EF4FA36
:100B70008327C4FB939727000327C4FCB307F70020
:100B8000032704FE23A0E700832784FE9387170032
:100B90002324F4FE832744FE938717002322F4FEC8
:100BA000832744FE0327C4FEE3E2E7F213000000BC
:100BB0008320C1050324810513010106678000001D
:100BC000130101FC232E1102232C810213040104C2
:100BD000232EA4FC232CB4FC232AC4FC2328D4FCFD
:100BE0002326E4FCB76702810327C4FD23A4E71E84
:100BF000B76702819387871E032784FD23A2E7003E
:100C0000B76702819387871E032744FD23A4E7006B
:100C1000B76702819387871E0327C4FC23A6E700DA
:100C2000B76702819387871E032704FD23A8E70087
:100C3000EFF0CFDC2324A4FE0327C4FC832784FE2B
:100C4000B357F7022326F4FE0327C4FC832784FE50
:100C5000B377F702638807008327C4FE93871700E2
:100C60002326F4FEB76702819387871E0327C4FEFD
:100C700023AAE7000327C4FC832784FE6362F702EC
:100C8000B76702819386871EB7170080138687CFC8
:100C9000832584FE032504FDEFF0CFFD6F000002E5
:100CA000B76702819386871EB7170080138687CFA8
:100CB0008325C4FC032504FDEFF0CFFBEFF08FD3B9
:100CC0002322A4FE032704FD832744FE63F8E700E4
:100CD000032544FEEFF01F896F00C000032504FDCB
:100CE000EFF05F88130000008320C1030324810319
:100CF0001301010467800000130101FB2326110486
:100D00002324810413040105232EA4FA232CB4FA0E
:100D1000EFF01F942320A4FE832704FE83A707007F
:100D2000232EF4FC832704FE83A74700232CF4FC26
:100D3000832704FE83A78700232AF4FC832704FE6D
:100D400083A747012326F4FE0327C4FE8327C4FBA1
:100D5000B307F7022324F4FE8327C4FE639A070037
:100D6000930710002326F4FE8327C4FB2324F4FEFC
:100D7000832704FE83A7C7002328F4FC232204FE54
:100D80006F00000C032784FB832704FD3307F70261
:100D9000832784FEB307F7002326F4FC032784FE91
:100DA000832704FDB337F70093F7F70F2324F4FCF0
:100DB000832784FC93B71700A303F4FC834774FCD8
:100DC000138F0700B7170080938FC7E26B200F00C7
:100DD0007B70FF018327C4FC939727000327C4FD82
:100DE000B307F70083A607008327C4FC9397270067
:100DF000032784FDB307F70003A707008327C4FC7C
:100E000093972700032644FDB307F6003387E600D7
:100E100023A0E700832784FE938717002324F4FE92
:100E2000B7170080138E07E367000E001300000061
:100E30006B300000832744FE938717002322F4FEC3
:100E4000832744FE0327C4FEE3EEE7F2130000000D
:100E50008320C1040324810413010105678000007D
:100E6000130101FC232E1102232C8102130401041F
:100E7000232EA4FC232CB4FC232AC4FC2328D4FC5A
:100E80002326E4FCB76702810327C4FD23A4E71EE1
:100E9000B76702819387871E032784FD23A2E7009B
:100EA000B76702819387871E032744FD23A4E700C9
:100EB000B76702819387871E0327C4FC23A6E70038
:100EC000B76702819387871E032704FD23A8E700E5
:100ED000EFF0CFB22324A4FE0327C4FC832784FEB3
:100EE000B357F7022326F4FE0327C4FC832784FEAE
:100EF000B377F702638807008327C4FE9387170040
:100F00002326F4FEB76702819387871E0327C4FE5A
:100F100023AAE7000327C4FC832784FE6362F70249
:100F2000B76702819386871EB7170080138687F9FB
:100F3000832584FE032504FDEFF0CFD36F0000026C
:100F4000B76702819386871EB7170080138687F9DB
:100F50008325C4FC032504FDEFF0CFD1EFF08FA96A
:100F60002322A4FE032704FD832744FE63F8E70041
:100F7000032544FEEFF00FDF6F00C000032504FDE2
:100F8000EFF04FDE130000008320C1030324810330
:100F90001301010467800000130101FB23261104E3
:100FA0002324810413040105232EA4FA232CB4FA6C
:100FB000EFF00FEA2320A4FE832704FE83A7070097
:100FC000232EF4FC832704FE83A74700232CF4FC84
:100FD000832704FE83A78700232AF4FC832704FECB
:100FE00083A747012326F4FE0327C4FE8327C4FBFF
:100FF000B307F7022324F4FE8327C4FE639A070095
:10100000930710002326F4FE8327C4FB2324F4FE59
:10101000832704FE83A7C7002328F4FC232204FEB1
:101020006F00000C032784FB832704FD3307F702BE
:10103000832784FEB307F7002326F4FC032784FEEE
:10104000832704FDB337F70093F7F70F2324F4FC4D
:10105000832784FC93B71700A303F4FC834774FC35
:10106000138F0700B7170080938FC70C6B200F00FA
:101070007B70FF018327C4FC939727000327C4FDDF
:10108000B307F70083A607008327C4FC93972700C4
:10109000032784FDB307F70003A707008327C4FCD9
:1010A00093972700032644FDB307F6003387E640F5
:1010B00023A0E700832784FE938717002324F4FEF0
:1010C000B7170080138E070D67000E001300000095
:1010D0006B300000832744FE938717002322F4FE21
:1010E000832744FE0327C4FEE3EEE7F2130000006B
:1010F0008320C104032481041301010567800000DB
:10110000130101FC232E1102232C8102130401047C
:10111000232EA4FC232CB4FC232AC4FC2328D4FCB7
:101120002326E4FCB76702810327C4FD23A0E72040
:10113000B767028193870720032784FD23A2E70076
:10114000B767028193870720032744FD23A4E700A4
:10115000B7670281938707200327C4FC23A6E70013
:10116000B767028193870720032704FD23A8E700C0
:10117000EFF0CF882324A4FE0327C4FC832784FE3A
:10118000B357F7022326F4FE0327C4FC832784FE0B
:10119000B377F702638807008327C4FE938717009D
:1011A0002326F4FEB7670281938707200327C4FE36
:1011B00023AAE7000327C4FC832784FE6362F702A7
:1011C000B767028193860720B717008013868723AD
:1011D000832584FE032504FDEFF0CFA96F000002F4
:1011E000B767028193860720B7170080138687238D
:1011F0008325C4FC032504FDEFF0CFA7EFE09FFF9C
:101200002322A4FE032704FD832744FE63F8E7009E
:10121000032544FEEFF00FB56F00C000032504FD69
:10122000EFF04FB4130000008320C10303248103B7
:101230001301010467800000130101FB2326110440
:101240002324810413040105232EA4FA232CB4FAC9
:10125000EFF00FC02320A4FE832704FE83A707001E
:10126000232EF4FC832704FE83A7470083A70700EF
:10127000232CF4FC832704FE83A78700232AF4FC95
:10128000832704FE83A747012326F4FE0327C4FE19
:101290008327C4FBB307F7022324F4FE8327C4FE8D
:1012A000639A0700930710002326F4FE8327C4FBEC
:1012B0002324F4FE832704FE83A7C7002328F4FC1D
:1012C000232204FE6F00000B032784FB832704FD09
:1012D0003307F702832784FEB307F7002326F4FCC5
:1012E000032784FE832704FDB337F70093F7F70F36
:1012F0002324F4FC832784FC93B71700A303F4FC96
:10130000834774FC138F0700B7170080938F07364D
:101310006B200F007B70FF018327C4FC939727008D
:101320000327C4FDB307F70083A607008327C4FC87
:1013300093972700032744FDB307F700032784FD95
:101340003387E60023A0E700832784FE93871700F6
:101350002324F4FEB7170080138E473667000E0073
:10136000130000006B300000832744FE93871700B2
:101370002322F4FE832744FE0327C4FEE3E6E7F4BA
:10138000130000008320C10403248104130101051C
:1013900067800000130101FC232E1102232C81021F
:1013A00013040104232EA4FC232CB4FC232AC4FC24
:1013B0002328D4FC2326E4FCB76702810327C4FD5D
:1013C00023A0E720B767028193870720032784FDC6
:1013D00023A2E700B767028193870720032744FD14
:1013E00023A4E700B7670281938707200327C4FC83
:1013F00023A6E700B767028193870720032704FD30
:1014000023A8E700EFE09FDF2324A4FE0327C4FC0A
:10141000832784FEB357F7022326F4FE0327C4FC78
:10142000832784FEB377F702638807008327C4FE0F
:10143000938717002326F4FEB7670281938707205E
:101440000327C4FE23AAE7000327C4FC832784FEE6
:101450006362F702B767028193860720B71700809F
:101460001386C74C832584FE032504FDEFF08F808F
:101470006F000002B767028193860720B7170080CC
:101480001386C74C8325C4FC032504FDEFE09FFEB3
:10149000EFE05FD62322A4FE032704FD832744FE4A
:1014A00063F8E700032544FEEFF0CF8B6F00C00028
:1014B000032504FDEFF00F8B130000008320C10310
:1014C000032481031301010467800000130101FB61
:1014D000232611042324810413040105232EA4FAD6
:1014E000232CB4FAEFF0CF962320A4FE832704FE2A
:1014F00083A70700232EF4FC832704FE83A747005D
:1015000083A70700232CF4FC832704FE83A787000E
:10151000232AF4FC832704FE83A747012326F4FE35
:101520000327C4FE8327C4FBB307F7022324F4FE7A
:101530008327C4FE639A0700930710002326F4FE56
:101540008327C4FB2324F4FE832704FE83A7C7005C
:101550002328F4FC232204FE6F00000B032784FBE6
:10156000832704FD3307F702832784FEB307F700C0
:101570002326F4FC032784FE832704FDB337F700FA
:1015800093F7F70F2324F4FC832784FC93B7170009
:10159000A303F4FC834774FC138F0700B717008084
:1015A000938F475F6B200F007B70FF018327C4FC84
:1015B000939727000327C4FDB307F70083A607000E
:1015C0008327C4FC93972700032744FDB307F70044
:1015D000032784FD3387E60223A0E700832784FEE8
:1015E000938717002324F4FEB7170080138E875FBC
:1015F00067000E00130000006B300000832744FEDC
:10160000938717002322F4FE832744FE0327C4FE9A
:10161000E3E6E7F4130000008320C10403248104FF
:101620001301010567800000130101FD23268102DB
:1016300013040103232EA4FC232604FE6F000001E3
:101640008327C4FE938717002326F4FE0327C4FED6
:101650008327C4FDE346F7FE130000000324C10204
:101660001301010367800000130101FD232611020D
:101670002324810213040103232EA4FC232CB4FC95
:10168000B7670281138787218327C4FDB307F7005B
:10169000130710002380E7008327C4FD6390070C25
:1016A000A30104FE232604FE6F00800A232604FE05
:1016B000232404FE6F004003B7670281138787214C
:1016C000832784FEB307F70083C7070063880700FA
:1016D0008327C4FE938717002326F4FE832784FE06
:1016E000938717002324F4FE032784FE832784FDB9
:1016F000E344F7FC0327C4FE832784FD631AF70441
:10170000232204FE6F000004B7670281138787213C
:10171000832744FEB307F70023800700B7970281B1
:10172000130710002380E72E13056004EFF0DFEFAE
:10173000B79702812380072E832744FE93871700E3
:101740002322F4FE032744FE832784FDE34EF7FAA9
:10175000834734FEE39C07F46F004002130000004F
:10176000B797028183C7072E93C7170093F7F70F28
:10177000E39807FE13054006EFF01FEB130000008F
:101780008320C1020324810213010103678000004A
:10179000130101FE232E810013040102232604FEFF
:1017A0006F008004B76702810327C4FE1317270068
:1017B00093878723B307F7001307300023A0E700C0
:1017C000B77702810327C4FE131727009387872367
:1017D000B307F7001307200023A0E7008327C4FE08
:1017E000938717002326F4FE0327C4FE9307F00F08
:1017F000E3DAE7FA130000000324C1011301010238
:1018000067800000130101FD2326110223248102B9
:1018100013040103232EA4FCB7070081138587114D
:10182000EFE05FFB232604FE6F0080058327C4FEE4
:10183000638E07008327C4FE93F7F70063980700C1
:10184000B70700811385C713EFE0DFF88327C4FED5
:10185000939727000327C4FDB307F70083A707006A
:1018600013850700EFE0DFFAB7070081138507143F
:10187000EFE05FF68327C4FE938717002326F4FE6C
:101880000327C4FE9307F00FE3D2E7FAB7070081FE
:1018900013854714EFE01FF4130000008320C102FA
:1018A000032481021301010367800000130101FF7B
:1018B000232611002324810013040101EFF05FEDC2
:1018C00093060001B787028113868723B7770281C9
:1018D00093858723B767028113858723EFF00F84F1
:1018E000B707008113858716EFE0DFEEB787028127
:1018F00013858723EFF01FF193070000138507007E
:101900008320C100032481001301010167800000CE
:02000004810079
:10000000300000003100000032000000330000002A
:10001000340000003500000036000000370000000A
:10002000380000003900000061000000620000009C
:10003000630000006400000065000000660000002E
:100040007761697420666F723A200000466F756EA2
:10005000643A20003000000031000000320000004F
:1000600033000000340000003500000036000000BE
:100070003700000038000000390000006100000077
:1000800062000000630000006400000065000000E2
:10009000660000000A00000030000000310000008F
:1000A0003200000033000000340000003500000082
:1000B0003600000037000000380000003900000062
:1000C00061000000620000006300000064000000A6
:1000D00065000000660000003000000031000000F4
:1000E0003200000033000000340000003500000042
:1000F0003600000037000000380000003900000022
:100100006100000062000000630000006400000065
:1001100065000000660000002D2D2D2D2D2D2D2DAC
:100120002D2D2D2D2D2D2D2D2D2D2D2D2D2D2D2DFF
:100130002D2D2D2D2D2D2D0A000000000A00000070
:10014000200000000A2D2D2D2D2D2D2D2D2D2D2D96
:100150002D2D2D2D2D2D2D2D2D2D2D2D2D2D2D2DCF
:100160002D2D2D2D0A0000000A0A4D617472697848
:10017000206D756C7469706C69636174696F6E0A67
:01018000007E
:100184000000008104000081080000810C0000814F
:100194001000008114000081180000811C000081FF
:1001A4002000008124000081280000812C000081AF
:1001B4003000008134000081380000813C0000815F
:1001C40054000081580000815C00008160000081BF
:1001D40064000081680000816C000081700000816F
:1001E40074000081780000817C000081800000811F
:1001F40084000081880000818C00008190000081CF
:10020400980000819C000081A0000081A40000816E
:10021400A8000081AC000081B0000081B40000811E
:10022400B8000081BC000081C0000081C4000081CE
:10023400C8000081CC000081D0000081D40000817E
:10024400D8000081DC000081E0000081E40000812E
:10025400E8000081EC000081F0000081F4000081DE
:10026400F8000081FC00008100010081040100818C
:10027400080100810C01008110010081140100813A
:040000058000000077
:00000001FF
